:1000000055C0000063C0000061C000005FC0000078
:100010005DC000005BC0000059C0000057C0000078
:1000200055C0000053C0000051C000004FC0000088
:100030004DC0000070C0000049C0000047C0000073
:1000400045C0000043C00000A9C000007DC0000002
:100050003DC000003BC0000039C0000037C00000B8
:1000600035C0000033C00000496D706F7274616E5E
:1000700074207461626C6520656E643A2030782566
:100080003032780A00496D706F7274616E7420743A
:1000900061626C65206265673A203078253032787D
:1000A0000A00746573742E2E2E0A000011241FBEE0
:1000B000CFEFD8E0DEBFCDBF21E0A0E0B1E001C0CE
:1000C0001D92A336B207E1F794D006C199CFCF9322
:1000D000C82F8A30C1F48DE0FADF80915C018F5F18
:1000E0008F7390915B019817E1F3E82FF0E0E55EE4
:1000F000FE4FC08380935C018091C1008062809339
:10010000C100CF9108958F3740F3CFE3E6CFDFDF13
:1001100090E080E008950F930FB70F930AB50F5F3B
:100120000ABD70F00BB50F4F0BBD50F000910001F0
:100130000F4F00930001009101010F4F0093010147
:100140000F910FBF0F9118951F920F920FB60F923C
:1001500011248F93EF93FF93E0915B01EF5FEF73B7
:10016000E0935B0180915C018E1305C08091C1001A
:100170008F7D8093C1008091C00080648093C00017
:10018000F0E0E55EFE4F80818093C600FF91EF9125
:100190008F910F900FBE0F901F9018951F920F9286
:1001A0000FB60F9211242F938F939F93EF93FF938A
:1001B0008091C0009091C600E0911A01EF5FE77056
:1001C000209119012E1799F08C71E0931A01F0E03B
:1001D000EF5EFE4F908380931001FF91EF919F910E
:1001E0008F912F910F900FBE0F901F90189582E066
:1001F000F2CF789483E084BD85BD81E080936F0069
:1002000094E09093B1008093B00087E880937A00E7
:100210001092C1001092800082E080938100559A74
:1002200095E195B99DE294B98093C0001092C50004
:1002300092E29093C40096E09093C20010925C0109
:1002400010925B0110921A01109219019091C10055
:1002500098699093C1009091C1009F7D9093C100D7
:1002600027E830E030930B0120930A0110920D0132
:1002700010920C018093050110920F0110920E0153
:1002800082E091E09093600180935F01C2EAD0E048
:10029000FE0184912196882311F019DFF9CFE0E760
:1002A000F8E0E4911F92EF9385E890E09F938F939D
:1002B00015D0E8E8F8E0E4911F92EF9388E690E02B
:1002C0009F938F930BD08DB79EB708960FB6F89477
:1002D0009EBF0FBE8DBFFFCFF894C8C2B0E0A0E0B4
:1002E000E3E7F1E09AC2AE01495F5F4FDA016D9139
:1002F0007D91AD010DE511E0F80182819381DC0172
:1003000013962C911397286013962C9309D0D8013B
:100310001296ED91FC912381277F2383E4E099C21B
:10032000ABE0B0E0E5E9F1E06AC27C013B018A01A3
:10033000FC0117821682838181FFBAC1CE0101962A
:100340005C01F7019381F30193FD859193FF819106
:100350003F01882309F449C1853239F493FD859121
:1003600093FF81913F01853221F4B70190E0B9D12B
:10037000E8CF912C212C312CFFE1F31538F08B3292
:1003800011F190F4803209F1833229F137FC3CC03D
:1003900020ED280F2A3050F536FE20C08AE0989EC6
:1003A000200D1124922E06C08D3291F0803371F70A
:1003B000689430F8F30193FD859193FF81913F019B
:1003C0008111DACF21C0689431F8689432F8F2CF05
:1003D000689433F8EFCF689434F8ECCFEAE02E9EBF
:1003E000200D1124222E689435F8E4CF8E3229F4A2
:1003F00036FCFBC0689436F8DDCF8C3619F468946F
:1004000037F8D8CF8836B1F2982F9F7D9554933026
:10041000D8F0833691F18337B1F1833509F05EC0AE
:100420002801F2E04F0E511CF801C080D180692DE7
:1004300070E036FC02C06FEF7FEFC6013CD14C018B
:10044000689437F882010AC00C5F1F4FFFE3F983FD
:1004500088248394912C6501E89437F833FE2AC0F0
:10046000522C8114910459F5552009F46ACFB70133
:1004700080E290E036D15A94F7CFF80180818983E9
:100480000E5F1F4FE5CF2801F2E04F0E511CF8011F
:10049000C080D180692D70E036FC02C06FEF7FEF25
:1004A000C60114D14C018201D7CFB70180E290E0A0
:1004B00018D12A942814190409F0B8F7D1CFF601FD
:1004C00037FC859137FE81916F01B70190E009D12A
:1004D00051105A94F1E08F1A9108C3CF843619F065
:1004E000893609F073C0F80137FE67C060817181F9
:1004F000828193810C5F1F4FF32DFF763F2E97FF74
:1005000009C090958095709561957F4F8F4F9F4F53
:10051000689437F82AE030E0A50113D1C82ECA1834
:100520008C2C432C36FE0CC0E89440F8C91440F4DF
:1005300034FE05C032FC03C0F32DFE7E4F2E892C05
:1005400044FE90C0FE01EC0DF11D8081803309F066
:1005500082C0242D297E422E842D8870582E43FC83
:100560008FC040FE89C09C2C821418F42C0C922C55
:10057000981844FE8BC0B70180E390E0B2D042FEF1
:1005800008C088E790E041FE02C088E590E0B7012E
:10059000A8D0C91408F486C0CA94D12C9FEFC91AF8
:1005A000D90ACA0CDB1CF60182916F01B70190E0F9
:1005B00098D0AC14BD04B9F757CF60817181072E74
:1005C000000C880B990B0E5F1F4F96CFD32CE8942D
:1005D000D4F82AE030E0853731F1232D297FD22E5F
:1005E0008F36F9F040F48835A1F0F70186819781C4
:1005F0002B96E2E120C1803749F08837B1F7D4FE6D
:1006000002C06894D2F820E130E00DC06894D4F8BC
:10061000F6CF34FE03C0822F8660D82E20E132E070
:1006200002C028E030E0F801D7FE0EC06081718181
:10063000828193810C5F1F4FA50183D0C82ECA18F9
:100640003D2CE89437F86CCF6081718190E080E0B8
:100650000E5F1F4FF1CF42FC02C083947DCF839485
:1006600083947ACF842D867809F476CFF6CFB701BC
:1006700080E290E036D083948214C8F3512C79CF75
:10068000522C5818821408F474CFF8CF842D867831
:1006900009F47FCF8BE241FE80E247FC8DE2B70197
:1006A00090E076CFB70180E390E01BD09A9471CFB1
:1006B0008FEF9FEF9DCFFC010590615070400110BE
:1006C000D8F7809590958E0F9F1F0895FC0161507B
:1006D000704001900110D8F7809590958E0F9F1F64
:1006E00008950F931F93CF93DF93182F092FEB01DA
:1006F0008B8181FD09C01FEF0FEF812F902FDF91BC
:10070000CF911F910F91089582FF14C02E813F81D8
:100710008C819D81281739073CF4E881F981CF014C
:1007200001969983888310838E819F8101969F8390
:100730008E83E3CFE885F985812F0995892BA1F375
:10074000DACFFA01AA27283051F1203181F1E8945B
:100750006F936E7F6E5F7F4F8F4F9F4FAF4FB1E0B4
:100760003ED0B4E03CD0670F781F891F9A1FA11DAF
:10077000680F791F8A1F911DA11D6A0F711D811DB0
:10078000911DA11D20D009F468943F912AE0269F75
:1007900011243019305D3193DEF6CF010895462FD4
:1007A0004770405D4193B3E00FD0C9F7F6CF462FB5
:1007B0004F70405D4A3318F0495D31FD405241931E
:1007C00002D0A9F7EACFB4E0A695979587957795DB
:1007D0006795BA95C9F700976105710508959B0162
:1007E000AC010A2E06945795479537952795BA95EB
:1007F000C9F7620F731F841F951FA01D08952F92C4
:100800003F924F925F926F927F928F929F92AF92A0
:10081000BF92CF92DF92EF92FF920F931F93CF93ED
:10082000DF93CDB7DEB7CA1BDB0B0FB6F894DEBF84
:100830000FBECDBF09942A88398848885F846E84AA
:100840007D848C849B84AA84B984C884DF80EE80F4
:10085000FD800C811B81AA81B981CE0FD11D0FB6FD
:10086000F894DEBF0FBECDBFED010895F894FFCF21
:10087000FFFFFFFFFFFFFFFFFFFFFFFFFFFFFFFF88
:09088000FFFFFFFFFFFFFFFFFF78
:00000001FF
